:1000000012C0189518951895189518951895189563
:100010001895189518951895189518951895189578
:100020001895189518958FE58DBFC0E1E8E84E2E1C
:1000300084E08EBFD4E0F3E05F2EEEEFF3E0A0E6C5
:10004000B0E088278D933197E9F789E189B980E09D
:1000500080BD88E18AB96624A09AA19AA29A8A9A58
:1000600085E086B980E487B9379AAAE6B0E08827A8
:100070008C9380E080939E0081E08093960080EDD9
:100080008093680081ED8093690078941FD520D813
:10009000A8E6B0E01C9133D817E031D810E12FD892
:1000A00025D888EE93E0F7D63AD5C7D6E2E7F1E156
:1000B000BED6C3D6C2D687D6082F013009F045C0B8
:1000C00086D6AAE6B0E08D9388278C93AAE6B0E0A6
:1000D000EEE8F1E1E5D709F001C0FFD0AAE6B0E013
:1000E000E0E9F1E1DDD709F007C035D5A6D6AAE6EB
:1000F000B0E088278C93DFCFAAE6B0E0E2E9F1E137
:10010000CFD709F001C00BD5AAE6B0E0E4E9F1E1F0
:10011000C7D709F009C081E0809396008ED6E6E942
:10012000F1E185D68AD689D6AAE6B0E0E0EBF1E126
:10013000B7D709F009C080E0809396007ED6E2EB45
:10014000F1E175D67AD679D601C03FD3D9D505D697
:10015000B2CFF894FFCFECECF1E169D66ED680E037
:100160008093970089E080939F0000919F00093A57
:1001700010F009F0AFC0A7E9B0E08C918F5F8C93CD
:100180005CD600919700013009F004C0EEEEF1E179
:100190004ED653D600919700023009F004C0E6E035
:1001A000F2E145D64AD600919700033009F004C029
:1001B000EEE1F2E13CD641D600919700043009F01F
:1001C00004C0E8E3F2E133D638D600919700053059
:1001D00009F004C0E4E5F2E12AD62FD6EEE6F2E11A
:1001E00026D62BD680E48093A40081E08093A000E3
:1001F0000091A000023110F009F060C00091A00051
:1002000041E00423A3EAB0E00C93A4EAB0E08C91AF
:100210008F5F8C93AFE9B0E08C918F5F8C93AFE9E7
:10022000B0E0EC91FF27A1EAB0E091E01CD7AFE984
:10023000B0E08C918F5F8C93AFE9B0E0EC91FF2739
:10024000A2EAB0E091E00FD7A4EAB0E08C91F8D533
:10025000E0E7F2E1ECD50091A1000A3008F003C01C
:10026000E4E7F2E1E4D5A0E7B3E0E1EAF0E056D656
:10027000D6D5E6E7F2E1DBD50091A2000A3008F01E
:1002800003C0E4E7F2E1D3D5A0E7B3E0E2EAF0E0AF
:1002900045D6C5D50091A300013009F004C0E8E7B8
:1002A000F2E1C5D504C0E2E8F2E1C1D5C6D5A0EAC5
:1002B000B0E08C918F5F8C9308F49ACFBED5EAE8BA
:1002C000F2E1B5D5BAD5AFE9B0E08C918F5F8C93F0
:1002D00008F44BCFB2D5089508953DDFECEAF2E182
:1002E000A6D5A2E6B0E08C91A0E7B3E0B3D597D550
:1002F000E2EBF2E19CD5A3E6B0E08C91A0E7B3E09D
:10030000A9D58DD5E2EBF2E192D5A4E6B0E08C91CF
:10031000A0E7B3E09FD583D5E4EBF2E188D5A7E66B
:10032000B0E08C91A0E7B3E095D579D5E6E7F2E1AE
:100330007ED5A6E6B0E08C91A0E7B3E08BD56FD573
:10034000E6E7F2E174D5A5E6B0E08C91A0E7B3E072
:1003500081D565D572D571D5E8EBF2E168D56DD55B
:10036000E6EEF2E164D569D5EAEFF2E160D565D554
:1003700064D5EEE2F3E15BD560D5E6E5F3E157D570
:100380005CD500E816E928E930E0A9EAB0E00D9371
:100390001D932D933C93E2E9F3E149D5AAE6B0E041
:1003A0003EE0F6D4AAE6B0E0E2ECF3E179D609F05B
:1003B00007C088E08093A400E4ECF3E138D53DD594
:1003C000AAE6B0E0E0EDF3E16BD609F007C08DE2FC
:1003D0008093A400E2EDF3E12AD52FD5AAE6B0E0A0
:1003E000EEEDF3E15DD609F007C082E58093A4004D
:1003F000E0EEF3E11CD521D5AAE6B0E0EEEEF3E1A4
:100400004FD609F007C087E78093A400E0EFF3E13F
:100410000ED513D5AAE6B0E0E0E0F4E141D609F04C
:1004200007C08CE98093A400E2E0F4E100D505D593
:10043000E0E1F4E1FCD4AAE6B0E03EE0A9D4AAE60B
:10044000B0E028D6A0E6B0E08C9381E0EAE6F0E0E8
:1004500001E00A93ABE8B0E0DDD5ABE8B0E08C9109
:10046000ABE9B0E08C930091A40041E0040FA5EA51
:10047000B0E00C9300919B00013481E008F480E02F
:100480008F9300919B00023581E010F009F080E02D
:100490009F918923882309F425C081E48093A800D3
:1004A0000091A800023510F009F01BC0A4EAB0E0EA
:1004B0008C918E5F8C930091A40041E0040FA5EA1B
:1004C000B0E00C934091A80000919B00041709F044
:1004D00001C007C0A8EAB0E08C918F5F8C9308F44C
:1004E000DFCF04C1043509F0FAC0AAE6B0E0D2D5E6
:1004F000082F0E3009F40EC0AAE6B0E088278C93CE
:10050000EEE3F4E194D499D4EEE6F4E190D495D4FA
:10051000D2CDE4C082E0EAE6F0E002E00A93A9E787
:10052000B0E078D5A9E7B0E043D5A2E6B0E00C93FF
:1005300084E0EAE6F0E002E00A93ACE7B0E06AD5D6
:10054000ACE7B0E035D5A3E6B0E00C9386E0EAE690
:10055000F0E002E00A93AFE7B0E05CD5AFE7B0E0CF
:1005600027D5A4E6B0E00C9389E0EAE6F0E002E0EB
:100570000A93A8E8B0E04ED5A8E8B0E019D5A7E600
:10058000B0E00C938BE0EAE6F0E002E00A93A5E825
:10059000B0E040D5A5E8B0E00BD5A6E6B0E00C93FE
:1005A0008DE0EAE6F0E002E00A93A2E8B0E032D59E
:1005B000A2E8B0E0FDD4A5E6B0E00C93A2E6B0E07E
:1005C0008C9153D4A2E6B0E08C93A3E6B0E08C917A
:1005D0004CD4A3E6B0E08C93A4E6B0E08C9145D473
:1005E000A4E6B0E08C93A5E6B0E08C913ED4A5E6FD
:1005F000B0E08C93A6E6B0E08C9137D4A6E6B0E0EC
:100600008C93A7E6B0E08C9130D4A7E6B0E08C9351
:100610005FD5A8E6B0E01C9172D510E070D5A5E6D4
:10062000B0E01C916CD5A6E6B0E01C9168D5A7E6B9
:10063000B0E01C9164D55AD54BD5A8E6B0E01C912A
:100640005ED514E05CD5A2E6B0E01C9158D5A3E6D7
:10065000B0E01C9154D5A4E6B0E01C9150D546D52D
:10066000ECE8F4E1E4D3A2E6B0E08C91A0E7B3E0DB
:10067000F1D3D5D3E2EBF2E1DAD3A3E6B0E08C918B
:10068000A0E7B3E0E7D3CBD3E2EBF2E1D0D3A4E62B
:10069000B0E08C91A0E7B3E0DDD3C1D3CED3EAE9DB
:1006A000F4E1C5D3A7E6B0E08C91A0E7B3E0D2D3E4
:1006B000B6D3E6E7F2E1BBD3A6E6B0E08C91A0E7C3
:1006C000B3E0C8D3ACD3E6E7F2E1B1D3A5E6B0E03E
:1006D0008C91A0E7B3E0BED3A2D3AFD307C0ECEABE
:1006E000F4E1A5D3AAD381E080939E0000919E00FF
:1006F000003081E009F080E08F93009160000430C9
:1007000080E010F009F081E09F918923882309F4AB
:1007100054C082E0EAE6F0E002E00A93ADE8B0E01F
:1007200079D4ADE8B0E044D4A1EAB0E00C9384E021
:10073000EAE6F0E002E00A93ADE8B0E06BD4ADE8A1
:10074000B0E036D4A2EAB0E00C93A4EAB0E0EC91B9
:10075000FF27A1EAB0E091E07BE774D4A5EAB0E01E
:10076000EC91FF27A2EAB0E091E07BE76BD4ABE825
:10077000B0E057D3E0E7F2E15AD30091A1000A308C
:1007800008F003C0E4E7F2E152D3A0E7B3E0E1EA06
:10079000F0E0C4D344D3E6E7F2E149D30091A200EC
:1007A0000A3008F003C0E4E7F2E141D3A0E7B3E088
:1007B000E2EAF0E0B3D333D340D380E080939E00ED
:1007C000AAE6B0E088278C93089582D4A8E6B0E02A
:1007D0001C9195D410E093D47BD4A9E6B0E01C9191
:1007E0008ED4ACD4A5E6B0E01C93A8D4A6E6B0E0C5
:1007F0001C93A4D4A7E6B0E01C93A0D4A1E6B0E07B
:100800001C939CD4A2E6B0E01C9398D4A3E6B0E07D
:100810001C9392D4A4E6B0E01C9368D40091960097
:10082000013009F03AC0A2E6B0E08C91A0E7B3E055
:1008300011D3F5D2E2EBF2E1FAD2A3E6B0E08C916B
:10084000A0E7B3E007D3EBD2E2EBF2E1F0D2A4E60B
:10085000B0E08C91A0E7B3E0FDD2E1D2E4EBF2E1AD
:10086000E6D2A7E6B0E08C91A0E7B3E0F3D2D7D20E
:10087000E6E7F2E1DCD2A6E6B0E08C91A0E7B3E0D7
:10088000E9D2CDD2E6E7F2E1D2D2A5E6B0E08C9192
:10089000A0E7B3E0DFD2C3D2D0D2A1E6B0E09C9112
:1008A000EAD2A7EAB0E08C9388EE93E0F4D2089500
:1008B000A7E6B0E09C91DFD2ACE9B0E08C93A6E66D
:1008C000B0E09C91D8D2ADE9B0E08C93A5E6B0E061
:1008D0009C91D1D2A6EAB0E08C93A1E6B0E09C91C5
:1008E000CAD2A7EAB0E08C930091A700073081E05C
:1008F00008F080E08F930091A700013080E010F0B5
:1009000009F081E09F918923882309F4DEC00091DA
:10091000A700023009F003C089E080939F00009196
:10092000A700033009F003C08EE280939F0000917E
:10093000A700043009F003C083E580939F00009175
:10094000A700053009F003C088E780939F0000915D
:10095000A700063009F003C08DE980939F0081E075
:100960008093A0000091A000023110F009F0ADC00A
:100970000091A00041E00423A3EAB0E00C93AFE9AA
:10098000B0E08C918F5F8C93AFE9B0E0EC91FF27E2
:10099000A1EAB0E091E067D3AFE9B0E08C918F5F5E
:1009A0008C93AFE9B0E0EC91FF27A2EAB0E091E0D0
:1009B0005AD340919C000091A100041781E009F0F6
:1009C00080E08F9340919D000091A200041781E088
:1009D00009F080E09F9189238F930091A30001305B
:1009E00081E009F080E09F9189238F930091A60018
:1009F000053081E008F080E09F918923882309F485
:100A000026C0E4ECF4E113D218D2A89A949AE8E054
:100A1000F0E01AD2E2EEF4E10AD20FD2E0E0F5E122
:100A200006D20BD2A8989498EFE2F0E00DD2E4EC55
:100A3000F4E1FDD102D2A89A949AE5E0F0E004D264
:100A4000E2EEF4E1F4D1F9D1A898949837C040913E
:100A50009C000091A100041781E009F080E08F93D1
:100A600040919D000091A200041781E009F080E010
:100A70009F9189238F930091A300003081E009F0BA
:100A800080E09F9189238F930091A600053081E03B
:100A900008F080E09F918923882309F40FC0EEE2DB
:100AA000F5E1C5D1CAD1A89A949AE8E0F0E0CCD19A
:100AB000EEE4F5E1BCD1C1D1A8989498A0EAB0E0E9
:100AC0008C918F5F8C9308F44DCF0895EEE6F5E19D
:100AD000AED1B3D1E6E9F5E1AAD1AFD1EEEBF5E1C4
:100AE000A6D1EAECF5E1A3D1E0EEF5E1A0D1A5D1E4
:100AF000EAEEF5E19CD1A0E7B3E0E4EFF5E1DAD16D
:100B00008ED1E8E0F6E193D198D1E4E1F6E18FD11E
:100B100094D1EEE6F5E18BD190D18FD108958DD1AE
:100B2000ECE3F6E184D189D188D1E0E5F6E17FD12B
:100B300084D1EAE6F6E17BD180D1E2E8F6E177D133
:100B40007CD1ECE9F6E173D178D1ECEBF6E16FD131
:100B500074D173D1089500E816E928E930E0A9EAD4
:100B6000B0E00D931D932D933C93E2EEF6E15FD13F
:100B700033E00CD1A0E7B3E01BD2A8E9B0E00C93BE
:100B800000919800003010F009F001C0B4C055D1B8
:100B900000919800013009F007C0EEEEF1E147D175
:100BA0004CD189E080939F0000919800023009F0B9
:100BB00007C0E6E0F2E13BD140D18EE280939F0096
:100BC00000919800033009F007C0EEE1F2E12FD167
:100BD00034D183E580939F0000919800043009F0A0
:100BE00007C0E8E3F2E123D128D188E780939F0092
:100BF00000919800053009F007C0E4E5F2E117D153
:100C00001CD18DE980939F00EEE6F2E110D115D161
:100C100080E48093A40081E08093A0000091A00074
:100C2000023110F009F060C00091A00041E00423FF
:100C3000A3EAB0E00C93A4EAB0E08C918F5F8C93B0
:100C4000AFE9B0E08C918F5F8C93AFE9B0E0EC91AD
:100C5000FF27A1EAB0E091E006D2AFE9B0E08C91C5
:100C60008F5F8C93AFE9B0E0EC91FF27A2EAB0E090
:100C700091E0F9D1A4EAB0E08C91E2D0E0E7F2E1B2
:100C8000D6D00091A1000A3008F003C0E4E7F2E1F9
:100C9000CED0A0E7B3E0E1EAF0E040D1C0D0E6E793
:100CA000F2E1C5D00091A2000A3008F003C0E4E7E9
:100CB000F2E1BDD0A0E7B3E0E2EAF0E02FD1AFD09F
:100CC0000091A300013009F004C0E8E7F2E1AFD0E1
:100CD00004C0E2E8F2E1ABD0B0D0A0EAB0E08C9181
:100CE0008F5F8C9308F49ACFA8D0EAE8F2E19FD006
:100CF000A4D0A3D004C0E8E0F7E199D09ED0089535
:100D00000091A700073081E008F080E08F93009108
:100D1000A700013080E010F009F081E09F91892365
:100D2000882309F401C0C4DD0091A700073081E0E9
:100D300008F080E08F930091A700013080E010F070
:100D400009F081E09F918923882309F403C0AA98C0
:100D5000A99A02C0A998AA9A089583E4806487B9E1
:100D6000AED0A9E9B0E08D939C93A9E9B0E00D91D4
:100D70001C91023652E0150708F006C0929AE8E18D
:100D8000F7E155D05AD001C092980895A0E7B3E09A
:100D900022D0803089F0883091F08D3039F03323C3
:100DA000B9F38D933A9563FE4BD0F2CF63FC04C048
:100DB0008DE046D08AE044D088278C93089540D0B7
:100DC00011973395E5CF81E05F9B882708958827A9
:100DD0005F9B089500C00F931F932F933F93AF9392
:100DE000BF93A9EAB0E00D911D912D913D915F9BBC
:100DF00001C00BC08827802B812B822B832B39F0DD
:100E00000150104020403040F2CF8CB101C0882703
:100E1000BF91AF913F912F911F910F910895A0E73E
:100E2000B3E08D91882311F00BD0FBCF089550D003
:100E3000802D11F005D0FBCF08958DE001D08AE020
:100E40005D9BFECF8CB9089588EE93E024D0319756
:100E5000D9F70895982F82958F70805D8D939F703C
:100E6000905D9D9388278C9308954AE0082F02D1C6
:100E70000295802B0895892F8F70905110F0865F16
:100E8000FCCF08953197F1F70895689462F80895BA
:100E9000E89462F80895EF93FF93EE27E82BE92B8F
:100EA00031F0E8EEF3E03197F1F70197D1F7FF91D8
:100EB000EF9108950DD00D920020E1F70895369A34
:100EC0003699FECF369A3699FECF84B195B1089502
:100ED000C895319600200895040F151F261F371F4F
:100EE0000895000F111F221F331F089500951095BC
:100EF000209530950F5F1F4F2F4F3F4F0895019161
:100F000010810EC001911191219130810BC001918E
:100F1000108117FF05C03FEF2FEF04C0008111279C
:100F20002227332737FF03C0E1DF8DE28D93CF9374
:100F3000DF93CF92DF92EF92AA24BB24CC24DD244E
:100F4000EE2440E2CAE0DD2755E093E38881890F73
:100F500087FD9F7083FD907F891B89935A95A9F720
:100F6000C0DFAA1CBB1CCC1CDD1CEE1C4A9551F733
:100F7000E894EFE0FF2782910ED0EB30E0F71EF00F
:100F800068948A2D0CD088278D93EF90DF90CF90B6
:100F9000DF91CF910895982F829501D0892F8F707E
:100FA000805D26F0803309F4089568948D93089548
:100FB00000271127222733271DD08A3328F48033B6
:100FC00018F005D015D0F9CF0EF490CF08958053C6
:100FD0008F93402F512F622F732F83DF82DF7CDFAF
:100FE00080DF8F919927080F191F291F391F089536
:100FF0008D910895E894FCDF8032E9F38B32D9F3C8
:101000008930C9F38D3211F46894F2CF089588279E
:101010008D93089509919191992351F08A95D9F76B
:10102000319781918D930A9519F08823D1F708950E
:10103000EECFE199FECFEEBBFFBB3196089591E074
:1010400001C092E07B3751F47FB7F894F2DF8D91C5
:101050008DBBE29AE19A9A95C9F77FBF77270895E9
:1010600091E001C092E0E5DFE09A8DB38D939A950F
:10107000D1F70895FF93881BF9E0001FFA9511F44A
:10108000FF910895881F841B18F4840F8894F5CF6E
:101090000894F3CF8FEF83959D919923E1F70895FD
:1010A000689401C0E894AF93BF938D9116F091912D
:1010B00002C00EDF902D891718F011F48823A9F7CC
:1010C000BF91AF910895AC98AD98A498A598089554
:1010D000A59AA49803D0A59801D0A49AEF93FF9362
:1010E000E1E0F0E0CFDEFF91EF910895A59AA49A98
:1010F000F5DFA5989D9BFECFF1DFA498EFCF089474
:10110000111F01C0110F69F0A59A18F40000A498EE
:1011100002C0A49A00C0E2DFA5989D9BFECFDEDF4F
:10112000F1CFA59AA498DADFA5989D9BFECFE8940D
:101130009C99689462F8D2CF089401C08894331FB8
:1011400011E0A59AA498CADFA5989D9BFECFC6DFA3
:1011500088949C990894111FA0F7A59A379510F4CC
:10116000A49801C0A49ABADFA5989D9BFECFB6DFD4
:101170000895204D6F6B796B6C6F7320736B616D8D
:101180006275746973207665696B6961200053002C
:101190005A0048002B00204C61696B6F20726F640D
:1011A000796D617320696A756E67746173200000E0
:1011B0002D00204C61696B6F20726F64796D6173D3
:1011C0002069736A756E6774617320002A2A2A2069
:1011D0002020536B616D627563696F206E75737447
:1011E0006174796D6169202020202A2A2A0020203C
:1011F000202020202020202020205069726D616452
:1012000069656E6973002020202020202020202086
:101210002020416E7472616469656E6973002020DC
:101220002020202020202020202054726563696126
:101230006469656E69730000202020202020202032
:10124000202020204B657476697274616469656E34
:101250006973000020202020202020202020202032
:1012600050656E6B74616469656E6973000000009F
:10127000203D200030003A002020494E20202D2023
:10128000200020204F55542000002A2A2A2A2A2AEA
:101290002A2A2A2A2A2A2A2A2A2A2A2A2A2A2A2AAE
:1012A0002A2A2A2A2A2A2A2A2A2A000054203D20C9
:1012B00000002F00202D2000204E756F2041206956
:1012C0006B69205220797261206C61696B726F6466
:1012D0007A696F20736B616D62656A696D6F206CEE
:1012E00061696B617300205420797261204441541C
:1012F000412D4C61696B6173000020506176697A01
:101300006479733A204130383030202B20454E54D8
:101310004552202A2A20536B616D62657320692033
:1013200070616D6F6B612030383A303000002044BE
:1013300061746F73206972206C61696B6F20666FD6
:10134000726D617461733A2064646D6D79792D6892
:10135000686D6D737300204E7573746174796D756B
:10136000206D656E6975206175746F6D6174697348
:101370006B616920697373696A756E677320706F3A
:101380002034302073656B756E647A69752E2E2E4D
:101390000000497665736B697465207361766169D5
:1013A000746573206469656E6F73206E756D657208
:1013B00069206E756F203120696B692035203E20D1
:1013C000000031005069726D616469656E69730077
:1013D0003200416E7472616469656E697300330036
:1013E0005472656369616469656E697300003400F5
:1013F0004B657476697274616469656E6973000027
:10140000350050656E6B74616469656E69730000C8
:10141000497665736B697465207261696465206ED5
:10142000756F204120696B69205220206972205815
:10143000585858206C61696B6120203E2000204282
:101440006C6F67692064756F6D656E79732061726A
:101450006261206E656976796B6F206A6F6B7320AD
:1014600061746E61756A696E696D61730000204513
:1014700052524F5220424C4F474153204441544F07
:101480005320464F524D4154415300004E41554A5E
:10149000412044415441203D20004E41554A415392
:1014A000204C41494B4153203D20000020424C4FED
:1014B000474153204441544F5320464F524D4154CD
:1014C0004153000020536B616D627574697320692C
:1014D0002070616D6F6B6120696A756E67746173EE
:1014E000000020536B616D62757469732069207010
:1014F000616D6F6B612069736A756E6774617300EB
:1015000050616B6172746F74696E616920736B6195
:101510006D62657320706F203533207365632E20F4
:1015200050616C61756B6974652E2E2E000020531E
:101530006B616D62757469732069732070616D6F82
:101540006B6F7320696A756E677461730000205356
:101550006B616D62757469732069732070616D6F62
:101560006B6F732069736A756E67746173002020F6
:101570002A2A2A2A2A2A2A2A2A2A2A2A2A2A2A2ACB
:101580002A2A2A2A2A2A2A2A2A2A2A2A2A2A2A2ABB
:101590002A2A2A2A2A0020202A20204175746F6DC9
:1015A0006174696E6973206D6F6B796B6C6F7320FA
:1015B000736B616D62757469732020202A0020208E
:1015C0002A20202020202020000020202056657284
:1015D0002E20312E303020416C666120202000000A
:1015E00020202020202020202A0020202A20202007
:1015F0002020200031322D32392D32303037203248
:10160000323A31383A333000202020202020202068
:1016100020202A0020202A2020202020202053754E
:101620006B757265204D617461732026204B696D66
:10163000202020202020202020202A002050616708
:10164000616C62696E6973206D656E69753A000040
:10165000202D2049736A756E677469206C61696B0F
:101660006F20726F64796D610000202B20496A75CC
:101670006E677469206C61696B6F20726F64796D3D
:101680006100204820526F6479746920706167613D
:101690006C62696E69206D656E697500205A205212
:1016A0006F6479746920736B616D627563696F2013
:1016B0006E7573746174796D7573000020532049E1
:1016C0006A756E67746920736B616D627563696FAB
:1016D000206E7573746174796D6F206D656E6975B8
:1016E00000005361766169746573206469656E6F8B
:1016F00073206E756D65726973206E756F20312071
:10170000696B692035203E00204C61696B61732054
:10171000626169676573690050616B6569737469BB
:10172000206C61696B726F647A696F2062617465A5
:0617300072696A6100000D
:00000001FF
